:060000000200260219684F
:03000B0002156675
:0100130032BA
:01001B0032B2
:03002300021908B7
:10002600C2AF121546121865121F89121E6AD2AF88
:030036000200398C
:100039007400120C191207E2120BACB403FA12176E
:100049004F7800791F7A197B167C167D167E197FE9
:100059001F7400121F097800791F7A167B157C130B
:100069007D157E167F1F7401121F09781F791B7A6F
:10007900117B007C1B7D1B7E1B7F1F7402121F09D5
:10008900781F791B7A1B7B1B7C007D117E1B7F1FD0
:100099007403121F09781079187A1C7B1E7C1C7D49
:1000A900187E107F007404121F091200BB121694E7
:1000B9008086121EDF740075F000121EF1900ED6B4
:1000C900120BDB9010FA740075F00912078170E2C7
:1000D90022121EDF740075F000121EF1900EE91253
:1000E9000BDB9011AE740075F002120781740122C6
:1000F900121EDF740075F000121EF1900EFC120B37
:10010900DB740075F013121EF17402121EB574012E
:1001190075F013121EF17403121EB5740175F00106
:04012900121EF19021
:10012D0010C4120BDB740175F00D121EF1E52F20BA
:10013D00E605900CD68003900DD6543F2323120B69
:10014D00DD120BACD5E007052F532F7F80D7D5E0FF
:10015D0007152F532F7F80CD740122121EDF7400DF
:10016D0075F000121EF1900F0F120BDB740075F07D
:10017D0013121EF17402121EB5740175F013121EC6
:10018D00F17403121EB5740175F001121EF1901079
:10019D00C4120BDB740175F00D121EF1E52A20E679
:1001AD0005900CD68003900DD6543F2323120BDD02
:1001BD00120BACD5E007052A532A7F80D7D5E0076F
:0301CD00152A539D
:1001D0002A7F80CD740222121EDF740075F0001297
:1001E0001EF1900F22120BDB9011D6740075F002F5
:1001F000120781741422121EDF740075F000121EA3
:10020000F1900F35120BDB9011FE740075F00212A5
:100210000781741522121EDF740075F000121EF1A2
:10022000900F5B120BDB740075F013121EF1740259
:10023000121EB5740175F013121EF17403121EB56F
:10024000740175F001121EF19010D6120BDB7401CF
:1002500075F00A121EF1E52B04120BF0120BACD54F
:10026000E007052B532B0F80E5D5E007152B532B0B
:070270000F80DB7415221260
:100277001EDF740075F000121EF1900F6E120BDB7B
:10028700740075F013121EF17402121EB574017515
:10029700F013121EF17403121EB5740175F00112EA
:1002A7001EF19010D6120BDB740175F00A121EF1C5
:1002B700E52C04120BF0120BACD5E007052C532CE0
:1002C7000F80E5D5E007152C532C0F80DB74152222
:1002D700121EDF740075F000121EF1900F48120B0A
:1002E700DB901226740075F0021207817416221231
:1002F7001EDF740075F000121EF1900F81120BDBE8
:10030700740075F013121EF17402121EB574017594
:08031700F013121EF174031231
:10031F001EB5740175F001121EF19010D6120BDB91
:10032F00740175F00A121EF1E52604120BF0120B80
:10033F00ACD5E007052653260F80E5D5E007152637
:10034F0053260F80DB741622121EDF740075F00027
:10035F00121EF1900F94120BDB740075F013121E26
:10036F00F17402121EB5740175F013121EF17403AD
:10037F00121EB5740175F001121EF19010D6120BFA
:10038F00DB740175F00A121EF1E52704120BF0124F
:10039F000BACD5E007052753270F80E5D5E00715F0
:1003AF002753270F80DB741622121EDF740075F09F
:0203BF0000122A
:1003C1001EF1900FA7120BDB90124E740075F00214
:1003D100120781741E22121EDF740075F000121EB6
:1003E100F1900FBA120BDB901276740075F00212C5
:1003F1000781741F22121EDF740075F000121EF1B6
:10040100900FE0120BDB740075F013121EF17402F1
:10041100121EB5740175F013121EF17403121EB58C
:10042100740175F001121EF19010E8120BDB7401DA
:1004310075F00C121EF1E52D120C01120BACD5E07A
:1004410008052DA2E692E780E5D5E008152DA2E684
:1004510092E780DA741F22121EDF740075F0001219
:0E0461001EF1900FF3120BDB740075F01312F6
:10046F001EF17402121EB5740175F013121EF17491
:10047F0003121EB5740175F001121EF19010E812EF
:10048F000BDB740175F00C121EF1E52E120C01122C
:10049F000BACD5E008052EA2E692E780E5D5E00883
:1004AF00152EA2E692E780DA741F22121EDF740067
:1004BF0075F000121EF1900FCD120BDB90129E748F
:1004CF000075F002120781742022121EDF7400756E
:1004DF00F000121EF1901006120BDB740075F01372
:1004EF00121EF17402121EB5740175F013121EF173
:1004FF007403121EB5740175F001121EF19010E80D
:0E050F00120BDB740175F00C121EF1E52812C0
:10051D000C01120BACD5E0080528A2E692E780E5A8
:10052D00D5E0081528A2E692E780DA742022121E83
:10053D00DF740075F000121EF1901019120BDB74B0
:10054D000075F013121EF17402121EB5740175F0D0
:10055D0013121EF17403121EB5740175F001121EF3
:10056D00F19010E8120BDB740175F00C121EF1E521
:10057D0029120C01120BACD5E0080529A2E692E771
:10058D0080E5D5E0081529A2E692E780DA742022ED
:10059D00121EDF740075F000121EF190102C120B5C
:1005AD00DB9012C6740075F00212078174282212B6
:1005BD001EDF740075F000121EF190103F120BDB60
:0605CD009012EE7400A282
:1005D30002B3340075F002120781742922D2027427
:1005E3002922C202742922121EDF740075F0001240
:1005F3001EF1901052120BDB9013167400A205B378
:10060300340075F002120781742A22D205742A225B
:10061300C205742A22121EDF740075F000121EF147
:10062300901065120BDB90133E7400A20F3400751B
:10063300F002120781743222C20F743322D20F7474
:100643003422121EDF740075F000121EF190107830
:10065300120BDB901366E53375F00A84142009024C
:10066300740575F00612078122D20975330A746185
:0206730022D291
:1006750009753314746222D20975331E746322D24C
:1006850009753328746422D209753332746522C220
:1006950009746622121EDF740075F000121EF190B7
:1006A500108B120BDB9013DE740075F008120781B6
:1006B5007446227400120C197447227401120C1925
:1006C5007448227402120C197449227403120C190D
:1006D500744A227404120C19744B227405120C19F5
:1006E500744C227406120C19744D227407120C19DD
:1006F500744E22121EDF740075F000121EF1901068
:100705009E120BDB90147E740075F008120781743D
:1007150050227400120C687451227401120C687412
:0D07250052227402120C68745322740312E5
:100732000C687454227404120C68745522740512E5
:100742000C687456227406120C68745722740712CD
:100752000C68745822121EDF740075F000121EF12C
:100762009010B1120BDB90151E740075F002120787
:1007720081745A22745B2274FF1219A0745C22FEE7
:10078200AFF0740075F012121EF17400121EB574EF
:1007920001121EB5740175F012121EF17402121EBE
:1007A200B57403121EB5740175F000121EF17404C3
:1007B200121EB5740175F001121EF1EE75F014A44B
:1007C200120BDD120BACD5E008EE75F014A4241167
:1007D20073D5E0090EEFB506DA7E0080D6740022EA
:1007E20012174F121F03780479047A047B047C04E5
:1007F2007D047E047F007400121F09780A790A7A48
:100802000A7B0E7C0A7D0A7E0A7F007401121F0990
:10081200780479047A0A7B0E7C0A7D0A7E0A7F00BC
:100822007402121F097804790A7A087B047C027D1B
:100832000A7E047F007403121F09780C790A7A0A6F
:100842007B0C7C0A7D0A7E0C7F007404121F0978DF
:1008520015790A7A157B0A7C157D0A7E157F0A7442
:1008620005121F09780A79157A0A7B157C0A7D150B
:100872007E0A7F157406121F0974192531C0E0E53E
:10088200874401F587D0E0B531F3740075F00412A6
:100892001EF17400121EB5740F2531C0E0E58744C5
:1008A20001F587D0E0B531F3740075F004121EF142
:1008B2007401121EB5740075F006121EF174001256
:1008C2001EB5740F2531C0E0E5874401F587D0E0FD
:1008D200B531F3740075F004121EF17448121EB59E
:1008E200740075F006121EF17402121EB5740075C2
:1008F200F008121EF17400121EB5740F2531C0E00B
:10090200E5874401F587D0E0B531F3740075F00650
:10091200121EF17441121EB5740075F008121EF118
:100922007403121EB5740075F00A121EF1740012DF
:100932001EB5740F2531C0E0E5874401F587D0E08C
:10094200B531F3740075F008121EF17453121EB51E
:10095200740075F00C121EF17400121EB5740F258E
:1009620031C0E0E5874401F587D0E0B531F374008A
:1009720075F00A121EF17449121EB5740075F00C5E
:10098200121EF17404121EB5740075F00E121EF1DF
:100992007400121EB5740F2531C0E0E5874401F5DD
:1009A20087D0E0B531F3740075F00C121EF1744279
:1009B200121EB5740075F00E121EF17402121EB5ED
:1009C200740F2531C0E0E5874401F587D0E0B531E9
:1009D200F3740075F00E121EF17441121EB5741EEE
:1009E2002531C0E0E5874401F587D0E0B531F374E5
:1009F2000175F00E121EF17447121EB574082531EE
:100A0200C0E0E5874401F587D0E0B531F3740175A4
:080A1200F00D121EF1744E12EA
:100A1A001EB574082531C0E0E5874401F587D0E0AA
:100A2A00B531F3740175F00C121EF17449121EB53A
:100A3A0074082531C0E0E5874401F587D0E0B53177
:100A4A00F3740175F00B121EF17452121EB574087C
:100A5A002531C0E0E5874401F587D0E0B531F3746C
:100A6A000175F00A121EF17445121EB5740825317B
:100A7A00C0E0E5874401F587D0E0B531F37401752C
:100A8A00F009121EF17445121EB574082531C0E032
:100A9A00E5874401F587D0E0B531F3740175F008B4
:100AAA00121EF1744E121EB574082531C0E0E58796
:100ABA004401F587D0E0B531F3740175F007121ED1
:100ACA00F17449121EB574082531C0E0E587440166
:100ADA00F587D0E0B531F3740175F006121EF17492
:100AEA0047121EB574082531C0E0E5874401F58731
:100AFA00D0E0B531F3740175F005121EF1744E128F
:100B0A001EB574082531C0E0E5874401F587D0E0B9
:100B1A00B531F3740175F004121EF17445121EB555
:100B2A0074082531C0E0E5874401F587D0E0B53186
:100B3A00F3740075F000121EF17405121EB57406E6
:100B4A00121EB57405121EB5740175F000121EF15D
:100B5A007405121EB57406121EB57405121EB574FC
:100B6A000075F010121EF17405121EB57406121EDD
:100B7A00B57405121EB5740175F010121EF17405D4
:100B8A00121EB57406121EB57405121EB5746425BC
:100B9A0031C0E0E5874401F587D0E0B531F312169C
:100BAA0094227801E5874401F587E2540370F5E55C
:100BBA00874401F587E2540360F574052531C0E0E6
:100BCA00E5874401F587D0E0B531F3E2540360DFED
:100BDA00227400F5F09354F8600BE5F093121EB5F9
:100BEA00E5F00480EE2275F00A842430121EB5E581
:100BFA00F02430121EB52230E708F404F5F0742D03
:100C0A008004F5F0742B121EB5E5F0120BF0225495
:100C1A0007232323FF121F92882B89260507EF1229
:100C2A001F92882C89270507EF121F92882D892881
:100C3A000507EF121F92882E89290507EF121F92C6
:100C4A00882F892A0507EF121F928833E9A2E092BA
:100C5A0002A2E19205A2E69209A2E7920F225407A4
:100C6A00232323FF121FFCEF121FDDA82BA926EF57
:100C7A00121FB60507EF121FDDA82CA927EF121FB6
:050C8A00B60507EF12A2
:100C8F001FDDA82DA928EF121FB60507EF121FDDD4
:100C9F00A82EA929EF121FB60507EF121FDDA82FE7
:100CAF00A92AEF121FB60507EF121FDDA833A20204
:100CBF0092E0A20592E1A20992E6A20F92E7F9EF64
:100CCF00121FB61220122243332000432333004455
:100CDF0033200044233300453320004633200046A1
:100CEF002333004733200047233300413320004193
:100CFF002333004833200043322000432332004483
:100D0F003220004423320045322000463220004674
:100D1F002332004732200047233200413220004166
:100D2F002332004832200043312000432331004456
:100D3F003120004423310045312000463120004648
:100D4F00233100473120004723310041312000413A
:100D5F00233100483120004320200043232000444A
:100D6F00202000442320004520200046202000465C
:100D7F00232000472020004723200041202000414E
:100D8F0023200048202000632020006323200064DC
:100D9F0020200064232000652020006620200066AC
:100DAF00232000672020006723200061202000619E
:100DBF00232000682020006331200063233100646A
:100DCF003120006423310065312000663120006638
:100DDF00233100673120006723310061312000612A
:100DEF002331006831200063322000632332006416
:100DFF003220006423320065322000663220006604
:100E0F0023320067322000672332006132200061F5
:100E1F0023320068322000633320006323330064E1
:100E2F0033200064233300653320006633200066CF
:100E3F0023330067332000672333006133200061C1
:100E4F0023330068332000633420006323340064AD
:100E5F00342000642334006534200066342000669B
:100E6F00233400673420006723340061342000618D
:100E7F002334006834200063352000632335006479
:100E8F003520006423350065352000663520006667
:100E9F002335006735200067233500613520006159
:100EAF002335006835200063362000632336006445
:100EBF003620006423360065362000663620006633
:100ECF0023360067362000484153494241204D499F
:100EDF004449204D45524745520053504C495420E8
:100EEF004B4559424F415244202020200053504C33
:100EFF004954204D49444920494E2031202020009B
:100F0F0053504C4954204D49444920494E203220DA
:100F1F0020200041535349474E204348414E4E45F0
:100F2F004C202020200041535349474E2043484135
:100F3F004E2E4D4944492E310041535349474E20BF
:100F4F004348414E2E4D4944492E32004153534997
:100F5F00474E2043482E494E2E312E5550520041B8
:100F6F00535349474E2043482E494E2E312E4C4F56
:100F7F00570041535349474E2043482E494E2E3276
:100F8F002E5550520041535349474E2043482E4946
:100F9F004E2E322E4C4F57005452414E53504F53FA
:100FAF0045202020202020202020005452414E5345
:100FBF00504F5345204D4944492E20312000545263
:100FCF00414E53504F5345204D4944492E20322016
:100FDF00005452414E53502E494E2E3120555050F1
:100FEF00455220005452414E53502E494E2E31201F
:100FFF004C4F57455220005452414E53502E494E9C
:10100F002E3220555050455220005452414E5350CD
:10101F002E494E2E32204C4F5745522000415353EC
:10102F0049474E20434F4E54524F4C4552202000BB
:10103F0041535349474E20434F4E54522E494E2E43
:10104F0031200041535349474E20434F4E54522EA7
:10105F00494E2E32200053595354454D2045584385
:10106F004C5553495645202000414354495645207D
:10107F0053454E53494E4720202020004C4F4144AA
:10108F00204F5054494F4E532020202020200053F2
:10109F00415645204F5054494F4E53202020202079
:1010AF002000524553455420455850414E44455217
:1010BF00203F20200053706C6974706F696E74202C
:1010CF003C2020203E20004368616E6E656C203C02
:1010DF0020203E20202020200053656D69746F6E04
:1010EF006573203C2020203E20200053706C6974D3
:1010FF00206B6579626F6172642020200200DA41F3
:10110F00737369676E204368616E6E656C20202073
:10111F000201D75472616E73706F736520202020A7
:10112F00202020200203B841737369676E20436F3C
:10113F006E74726F6C65722002059D5379737465BE
:10114F006D204578636C75736976652002061841CA
:10115F0063746976652053656E73696E672020200E
:10116F000206454C6F6164206F7074696F6E732057
:10117F002020202002069953617665206F707469D4
:10118F006F6E7320202020200206F852657365745D
:10119F0020457870616E6465722020200207574DDC
:1011AF0049444920494E2031202020202020202052
:1011BF000200F94D49444920494E20322020202079
:1011CF00202020200201684D49444920494E2031FA
:1011DF0020202020202020200201F64D49444920C4
:1011EF00494E203220202020202020200202D755D7
:1011FF00707065722073656374696F6E2020202094
:10120F000202154C6F7765722073656374696F6E98
:10121F00202020200202765570706572207365635E
:10122F0074696F6E202020200202F64C6F77657272
:10123F002073656374696F6E202020200203574D61
:10124F0049444920494E20312020202020202020B1
:10125F000203D74D49444920494E203220202020F7
:10126F00202020200204BA557070657220736563C8
:10127F0074696F6E202020200203F64C6F77657221
:10128F002073656374696F6E202020200204585507
:10129F00707065722073656374696F6E20202020F3
:1012AF000204D94C6F7765722073656374696F6E32
:1012BF002020202002053B4D49444920494E203132
:1012CF0020202020202020200205BC4D4944492009
:1012DF00494E203220202020202020200205EA74B1
:1012EF006F2075707065722073656374696F6E20FF
:1012FF000205E0746F206C6F7765722073656374FD
:10130F00696F6E200205E5746F207570706572202D
:10131F0073656374696F6E2002060E746F206C6FB5
:10132F007765722073656374696F6E2002061345CB
:10133F0078636C757369766520202020202020202B
:10134F0002063B49676E6F72652020202020202007
:10135F00202020200206403130306D7320202020C5
:10136F00202020202020202002066C3230306D7388
:10137F00202020202020202020202020020674332F
:10138F0030306D732020202020202020202020208E
:10139F0002067C3430306D73202020202020202046
:1013AF00202020200206843530306D73202020202D
:1013BF00202020202020202002068C6F666620200F
:1013CF0020202020202020202020202002069446AC
:1013DF00696C65202330202844656661756C74291B
:1013EF000206B846696C652023312020202020207A
:1013FF00202020200206C046696C65202332202061
:10140F0020202020202020200206C846696C65205D
:10141F002333202020202020202020200206D04609
:10142F00696C6520233420202020202020202020BC
:10143F000206D846696C6520233520202020202005
:10144F00202020200206E046696C652023362020EC
:10145F0020202020202020200206E846696C6520ED
:10146F002337202020202020202020200206F04695
:10147F00696C65202330202844656661756C74297A
:10148F0002071746696C6520233120202020202079
:10149F002020202002071F46696C65202332202060
:1014AF00202020202020202002072746696C65205D
:1014BF0023332020202020202020202002072F4609
:1014CF00696C65202334202020202020202020201C
:1014DF0002073746696C6520233520202020202005
:1014EF002020202002073F46696C652023362020EC
:1014FF00202020202020202002074746696C6520ED
:10150F0023372020202020202020202002074F4E8C
:10151F004F2C20646F6E27742072657365742020C2
:10152F000207764F4B202020202020202020202033
:07153F0020202020020779A3
:1015460075331ED209C28C753000753100E5895499
:10155600F04401F589758AF0758CD8D28CD2A9220F
:10156600758AF5758CD8C0E0C0F0C0D0053105305D
:10157600E530B4646275300030085C740075F003C1
:10158600121EF1E53960077403121EB5800574005A
:10159600121EB5753900E53860077404121EB58051
:1015A600057400121EB5753800740175F003121E1D
:1015B600F1E53C60077403121EB580057400121E27
:1015C600B5753C00E53B60077404121EB5800574D2
:1015D60000121EB5753B0030091BC2AFE53D700D0C
:0E15E6001532E532700A74FE1219A0800385DA
:1015F4003332D2AF753D00300840E531540FB40F9B
:101604006EB20A901755200A33740075F005121E45
:10161400F1E53A932535F535E537932534753400EE
:1016240013C313C39408F40475F008901855F536E1
:1016340093121EB5E53604D5F0F4804D740175F0AF
:1016440005121EF1E537932534F534E53A93253533
:1016540075350013C313C39408F40475F008901887
:1016640055F53693121EB5E53604D5F0F4801AB458
:091674000717901755E53793257F
:10167D0034F534E53A932535F535753700753A006F
:10168D00D0D0D0F0D0E032780079007A007B007CA9
:10169D00007D007E007F007400121F09781F791FE6
:1016AD007A1F7B1F7C1F7D1F7E1F7F007401121F01
:1016BD0009781F79047A1F7B007C117D117E0E7FC6
:1016CD00007402121F09780479067A057B057C04E3
:1016DD007D1C7E187F007403121F097800790E7A25
:1016ED00157B177C117D0E7E007F007404121F097F
:1016FD00780E79047A047B047C047D047E0E7F00D1
:10170D007405121F09781F790A7A0A7B0A7C0A7DF3
:10171D000A7E1F7F007406121F09121EDF7402124B
:10172D001EB57405121EB5740175F000121EF1740C
:10173D0002121EB57406121EB5753400753500D231
:10174D000822C208121EDF22000102020303030356
:10175D000404040404040404050505050505050534
:10176D000505050505050505060606060606060614
:10177D0006060606060606060606060606060606FC
:10178D0006060606060606060707070707070707E4
:10179D0007070707070707070707070707070707CC
:1017AD0007070707070707070707070707070707BC
:1017BD0007070707070707070707070707070707AC
:1017CD000707070707070707080808080808080894
:1017DD00080808080808080808080808080808087C
:1017ED00080808080808080808080808080808086C
:1017FD00080808080808080808080808080808085C
:10180D00080808080808080808080808080808084B
:10181D00080808080808080808080808080808083B
:10182D00080808080808080808080808080808082B
:10183D00080808080808080808080808080808081B
:10184D000808080808080808010101010101010143
:08185D00000000000000000083
:10186500753F00754000753E007542007543007573
:101875004100754400754500C29B753700753800F9
:10188500754700754900752B00752C01752D007580
:101895002E00752F00753A00753B00754600754A98
:1018A50000752609752702752800752900752A0017
:0B18B500C200C201D202C203C204D272
:1018C00005753D00754800D20F759840E589540FA5
:1018D0004420F589E587C2E7F587758DFFC2ABD255
:1018E000ACD28ED29C78017400F27480F27400F253
:1018F00078007443F27480F2740EF278017458F236
:101900007404F2D288D2A822C2ACC0E0C000C0D019
:1019100030982DE53F2450F8E599C298B4FE0405AF
:10192000398014B4F8040538800DF6053E053F53A0
:101930003F0F05371219C0D0D0D000D0E0D2AC3262
:10194000C3E545B5440DC299C29BD0D0D000D0E0CC
:10195000D2AC322470F88699054553450FC299D010
:10196000D0D000D0E0D2AC32C2A8C0E0C000C0D01D
:101970007800E2B4FE04053C801DB4F804053B8009
:1019800016C0E0E5422460F8D0E0F6054105425378
:10199000420F053A121C14D0D0D000D0E0D2A832A9
:1019A000C2AC053D209B07F599D29BD2AC22C0E08A
:0319B0007470252B
:1019B30044F8D0E0F6054453440FD2AC22C2AF3012
:1019C3000403D2AF22200114E5402450F8E620E7B7
:1019D30003021A1D54F0B4F02D021AD0D2AFE6124E
:1019E30019A0054053400F153E20000E1549E54947
:1019F3006003021C0CC201021BF9B4F7F5C200C25A
:101A030001D2AF021BF9B4B003021BB15003021B96
:101A130056B4E003021BB1021BD5E547B4B0004046
:101A23006354F0B4B002802FB4E002802AE547B5D6
:0E1A33004810E61219A0D2AF054053400F151F
:101A41003E021BF9F5481219A0E61219A0D2AF0502
:101A51004053400F153E021BF9D201D2AF75490127
:101A6100E547B5480EE61219A0054053400F153E53
:101A7100021BF9F5481219A0E61219A005405340BE
:101A81000F153E021C0CD201D2AF754901E5475436
:101A9100F0C0E0E6054053400F153EB52F00400E63
:011AA100251F
:101AA2002D547FF8D0E0452BB54815800C252E54D7
:101AB2007FF8D0E0452CB54807E81219A0021C0CAB
:101AC200F547F5481219A0E81219A0021C0CE6B459
:101AD200F203021B26B4F303021B3EB4F003021B03
:101AE20007B4F70ED2AFC200054053400F153E02B5
:101AF2001BF9D2AF054053400F153EF547F548128A
:0F1B020019A0021BF9D200054053400F153E20D9
:101B11000F0ED201D2AFF547F5481219A0021C0CE5
:101B2100D2AF021C0CD201D2AF054053400F153E7B
:101B3100F547F5481219A0754902021C0CD201D2D1
:101B4100AF054053400F153EF547F5481219A075F2
:101B51004901021C0CE53EB40103D2AF22D201D2ED
:101B6100AF754901054053400F153EE654F0C0E002
:031B710074502588
:101B740040F8E6054053400F153EB52F00401725A9
:101B84002D547FF8D0E0452BF547F5481219A0E80D
:101B94001219A0021C0C252E547FF8D0E0452CF518
:101BA40047F5481219A0E81219A0021C0CD201D260
:101BB400AF054053400F153EE654F0200204452C77
:101BC4008002452BF547F5481219A0754902021CFD
:061BD4000CD201D2AF05A6
:101BDA004053400F153EE654F0200204452C800283
:101BEA00452BF547F5481219A0754901021C0CC28C
:101BFA00AFE5416003021C14D2AFE53E600302194F
:101C0A00C022E53E60030219DF22C2AF300103D2CF
:101C1A00AF22200414E5432460F8E620E703021CFF
:101C2A007154F0B4F02D021D26D2AFE61219A005A8
:101C3A004353430F154120030E154AE54A60030238
:051C4A001E62C204024D
:101C4F001E4FB4F7F5C203C204D2AF021E4FB4B099
:101C5F0003021E075003021DACB4E003021E07026D
:101C6F001E2BE546B4B000406554F0B4B002802F8F
:101C7F00B4E002802AE546B54810E61219A0D2AFAB
:101C8F00054353430F1541021E4FF5481219A0E6A5
:101C9F001219A0D2AF054353430F1541021E4FD265
:101CAF0004D2AF754A01E546B5480EE61219A005F4
:0A1CBF004353430F1541021E4FF579
:101CC900481219A0E61219A0D2AF054353430F15C4
:101CD90041021E62D204D2AF754A01E54654F0C0F2
:101CE900E0E6054353430F1541B52A00400E252868
:101CF900547FF8D0E04526B54815800C2529547F36
:101D0900F8D0E04527B54807E81219A0021E62F588
:101D190046F5481219A0E81219A0021E62E6B4F2AB
:101D290003021D7CB4F303021D94B4F003021D5D8C
:0A1D3900B4F70ED2AFC20305435306
:101D4300430F1541021E4FD2AF054353430F1541B5
:101D5300F546F5481219A0021E4FD203054353431B
:101D63000F1541200F0ED204D2AFF546F5481219D4
:101D7300A0021E62D2AF021E62D204D2AF05435349
:101D8300430F1541F546F5481219A0754A02021E84
:081D930062D204D2AF054353F4
:101D9B00430F1541F546F5481219A0754A01021E6D
:101DAB0062E541B40103D2AF22D204D2AF754A012E
:101DBB00054353430F1541E654F0C0E074602543CF
:101DCB00F8E6054353430F1541B52A004017252864
:101DDB00547FF8D0E04526F546F5481219A0E812D5
:101DEB0019A0021E622529547FF8D0E04527F5463D
:0A1DFB00F5481219A0E81219A00221
:101E05001E62D204D2AF054353430F1541E654F089
:101E1500200504452780024526F546F5481219A0F8
:101E2500754A02021E62D204D2AF054353430F1511
:101E350041E654F0200504452780024526F546F580
:101E4500481219A0754A01021E62C2AFE53E600341
:101E55000219C0D2AFE5416003021C1422E54160BE
:051E650003021C332202
:101E6A00C295C296C293C292D291D290D29400C223
:101E7A0094740A121F37D29400C2947401121F3745
:101E8A00D29400C2947401121F37C290D29400C235
:101E9A00947401121F377428121F5F740E121F5F89
:101EAA007401121F5F7406121F5F22121F44D2961A
:101EBA00C295339293339292339291339290D29401
:101ECA0000C294339293339292339291339290D286
:101EDA009400C294227401121F5F121EEB121F0398
:101EEA00227402121F5F226002744025F04480129D
:101EFA001F5F22740E121F5F22740C121F5F2223AF
:101F0A0023234440121F5FE8121EB5E9121EB5EAE8
:101F1A00121EB5EB121EB5EC121EB5ED121EB5EE71
:101F2A00121EB5EF121EB54480121F5F2275F0C84B
:101F3A00000000D5F0FAD5E0F422D293D292D291E1
:101F4A00D290D295C296D294A293C29400D294000F
:101F5A00C29440F222121F44C296C295339293331E
:101F6A009292339291339290D29400C29433929384
:0F1F7A00339292339291339290D29400C2942278
:101F8900C297C2B4C2B5D2B322543F4480C2B5C2CB
:101F9900B4D297C0E0D312206CD0E012207E122078
:101FA90089F8122089F9C2B5C2B4C29722543F44B4
:101FB90040C2B5C2B4D297C0E0D312206CD0E012AF
:101FC900207EE812207EE912207EC2B5C2B4C297F3
:101FD90012206222543F44C0C2B5C2B4D297C0E0B5
:101FE900D312206CD0E012207EC2B5C2B4C29712BF
:101FF900206222C2B5C2B4D297D312206C743012B7
:10200900207EC2B5C2B4C29722C2B5C2B4D297D398
:1020190012206C740012207EC2B5C2B4C29722C2CB
:10202900B5C2B4D297D312206C742012207EC2B5E7
:10203900C2B4C29712206222C2B5C2B4D297D312D7
:10204900206C741012207EE812207EE912207EC2D4
:10205900B5C2B4C29712206222D29700A2B350FC33
:10206900C2972292B4D2B500C2B522C2B4D2B50089
:10207900C2B5A2B32275F0083312206CD5F0F9224B
:0B20890075F00812207433D5F0F92226
:00000001FF
